:020000040000FA
:1000000064002500110A0A0281000307090AEA01B7
:100010000008EA01E8030D0AA902EC03100AAD0288
:100020000008000C26000F0C0200FC0C0600070C58
:1000300024006000A4024307190A61008607240A0D
:100040002606240A0705250A070403090B062E0ABB
:1000500027072E0A680069002B0526052B073A0A98
:10006000B70C89004307360A1B0C880003073A0ABD
:100070002B04260427073E0A0B053F0A0B0403093D
:10008000A607460A2607460A4705470A4704030902
:1000900047064E0A06064E0A27044F0A270503099B
:1000A0002E065A0A0E06640A0707640A6C006D00E1
:1000B0002E0506051E0C8D004307600A840C8C007B
:1000C0000307640A2E0406040707680A0E05690A76
:0600D0000E0403091E0AE4
:0203FE00000CF1
:080400000000010000000000F3
:021FFE00FA0FD8
:00000001FF
